:100000000C9483000C94132B0C943E2B0C94692BB2
:100010000C94AD000C94AD000C94AD000C94AD00AC
:100020000C94AD000C94AD000C94AD000C94AD009C
:100030000C94AD000C94AD000C94AD000C94AD008C
:100040000C94AD000C94AD000C942E290C94AD00D2
:100050000C9440270C9476270C94AD000C94AD00C2
:100060000C94AD000C94AD000C94AD000C94AD005C
:100070000C94AD000C94AD000C94AD000C94A20D4A
:100080000C94AD000C94AD000C94AD000000000188
:100090000200090A00000000040308070000000035
:1000A0000000000000000000000000000102040841
:1000B0001020408001020408102040800102040842
:1000C0001020408001020408102040800202020239
:1000D00002020202040404040404040403030303EC
:1000E00003030303010101010101010100002200DA
:1000F000250028002B0000002100240027002A00F2
:10010000C6055225AA2711241FBECFEFD0E4DEBFBB
:10011000CDBF11E0A0E0B1E0E0E4FFE500E00BBFFF
:1001200002C007900D92AA34B107D9F72CE3AAE4D4
:10013000B1E001C01D92AA32B207E1F710E0C3E8B6
:10014000D0E004C02197FE010E94D92DC038D1070C
:10015000C9F70E94D8270C949E2F0C940000FC0134
:100160002FB7F894A681B7816D937C934681578110
:10017000828193814817590731F480819181978357
:1001800086832FBF0895868197810296F8CF1F93AB
:10019000CF93DF93EC01162F0E94802F181739F0B0
:1001A000612FCE01DF91CF911F910C94882FDF91A9
:1001B000CF911F9108950C94802FDC01ED91FC915B
:1001C0000190F081E02D099461E08CE00C949E2A6E
:1001D00060E08CE00C949E2A61E08DE00C949E2AF5
:1001E00060E08DE00C949E2A0F931F93CF93DF93D2
:1001F0008C01EC01892B11F4C1E0D0E01C161D0626
:100200000CF561E08CE00E949E2A60E08DE00E9487
:100210009E2A64E670E080E090E00E94A92960E0F8
:100220008CE00E949E2A61E08DE00E949E2A64E696
:1002300070E080E090E00E94A92901151105F1F21B
:100240002197DCCF60E08CE00E949E2A60E08DE088
:10025000DF91CF911F910F910C949E2A0F931F93C2
:10026000CF93DF938C01EC01892B11F4C1E0D0E036
:1002700061E08DE00E949E2A60E08DE01C161D0664
:10028000BCF40E949E2A64E670E080E090E00E9448
:10029000A92961E08DE00E949E2A64E670E080E07A
:1002A00090E00E94A9290115110531F32197E4CFAF
:1002B000DF91CF911F910F910C949E2A0F931F9362
:1002C000CF93DF938C01EC01892B11F4C1E0D0E0D6
:1002D00060E08CE01C161D06BCF40E949E2A64E6B9
:1002E00070E080E090E00E94A92961E08CE00E942B
:1002F0009E2A64E670E080E090E00E94A929011542
:10030000110531F32197E4CFDF91CF911F910F9128
:100310000C949E2A8091423790914337A0914437A4
:10032000B09145370196A11DB11D8093423790933E
:100330004337A0934437B09345374091040150911F
:1003400005016091060170910701481759076A0776
:100350007B0720F5109242371092433710924437B2
:10036000109245376091473780910901861780F0D8
:1003700081E08093463780914637680F6093473716
:1003800070E08CE00E94B22B60E08DE00C949E2A1D
:1003900080910801681778F38FEFEBCF0895809173
:1003A000423790914337A0914437B0914537019639
:1003B000A11DB11D8093423790934337A0934437DA
:1003C000B0934537409104015091050160910601B9
:1003D00070910701481759076A077B0720F51092AB
:1003E000423710924337109244371092453760914C
:1003F000473780910901861780F081E08093463766
:1004000080914637680F6093473770E08DE00E9417
:10041000B22B60E08CE00C949E2A80910801681752
:1004200078F38FEFEBCF089560EC70E080E89BE30A
:100430000E94DD0066E070E080E89BE30E94DD0042
:100440006091533B70E080E89BE30E94DD0060EC2C
:1004500070E080E89BE30C94DD0060EC70E080E8E5
:100460009BE30E94DD0067E070E080E89BE30E9470
:10047000DD006091150170E080E89BE30E94DD00E3
:1004800060EC70E080E89BE30C94DD0060EC70E0D1
:1004900080E89BE30E94DD006FE070E080E89BE372
:1004A0000E94DD0061E070E080E89BE30E94DD00D7
:1004B00060EC70E080E89BE30C94DD0060EC70E0A1
:1004C00080E89BE30E94DD006FE070E080E89BE342
:1004D0000E94DD0070E060E080E89BE30E94DD00A8
:1004E00060EC70E080E89BE30C94DD0060EC70E071
:1004F00080E89BE30E94DD006EE070E080E89BE313
:100500000E94DD008091513B61E070E0811102C0EA
:1005100070E060E080E89BE30E94DD0060EC70E04A
:1005200080E89BE30C94DD0060EC70E080E89BE3E6
:100530000E94DD0068E070E080E89BE30E94DD003F
:1005400066E470E080E89BE30E94DD0060EC70E010
:1005500080E89BE30C94DD0060EC70E080E89BE3B6
:100560000E94DD0060E570E080E89BE30E94DD0012
:1005700061E070E080E89BE30E94DD006EE070E0E7
:1005800080E89BE30E94DD0060EC70E080E89BE384
:100590000C94DD008091533B882341F060915C3BDB
:1005A00070915D3B8EE59BE30C948F2308958091C1
:1005B000533B882341F060911801709119018EE539
:1005C0009BE30C94682408958091533B8823E1F0C9
:1005D0008091503B843A51F460911601709117015B
:1005E00050E040E08EE59BE30E9436258091503B31
:1005F000893A51F4609116017091170141E050E081
:100600008EE59BE30C94362508958091533B882317
:1006100061F08EE59BE30E9461216093583B7093EB
:10062000593B80935A3B90935B3B08958091533B99
:10063000882371F04091583B5091593B60915A3B4F
:1006400070915B3B8EE59BE30E94CE230C940503E7
:1006500008958091533B882361F08EE59BE30E94CF
:1006600031216093543B7093553B8093563B90935C
:10067000573B08958091533B882371F04091543B40
:100680005091553B6091563B7091573B8EE59BE3F3
:100690000E949D220C94290308958091533B882346
:1006A00021F08EE59BE30C94B02180E0089583ED6A
:1006B0009FE00E94DB0091E0833709F090E0892FF2
:1006C0000895C8E3DFE06FEFCE010E94C7002196D6
:1006D000C11580E1D807B9F70E94EC000E94E8003C
:1006E000FBCF88E39FE00E94DB0091E0833009F0BC
:1006F00090E0892F089589E39FE00E94DB00982F06
:100700008093503B81E0943A21F0993A11F080E0D7
:10071000089508958AE39FE00E94DB0080934F3B99
:100720009FEF980F81E09E3F08F080E00895BF9210
:10073000CF92DF92EF92FF920F931F93CF93DF93AD
:100740008BE090E00E9409287C018C01C8E3DFE087
:10075000CE010E94DB00F80181938F012196C33402
:10076000FFE0DF07A9F76BE070E0C7010E94CF1F31
:10077000B82EC92E082F192FDD24D394CE010E9444
:10078000DB00F80191918F018913D12C2196C3359B
:10079000FFE0DF0799F78B2D9C2D0E94A528C7014C
:1007A0000E94A5288D2DDF91CF911F910F91FF9071
:1007B000EF90DF90CF90BF9008958FED9FE00E9463
:1007C000DB0091E0833709F090E0892F0895CF9204
:1007D000DF92EF92FF92CF930E94DD03882309F40A
:1007E00061C084ED9FE00E94DB0090E090935D3B50
:1007F00080935C3B85ED9FE00E94DB0090E090934E
:1008000019018093180186ED9FE00E94DB0090E0C3
:1008100090931701809316018BED9FE00E94DB00FF
:10082000C82F8CED9FE00E94DB0090E0B0E0A0E0DC
:100830007C01DD24CC24FC2A8DED9FE00E94DB00AE
:10084000C82F8EED9FE00E94DB00C82ADC2AC092F0
:10085000543BD092553BE092563BF092573B87ED8C
:100860009FE00E94DB00C82F88ED9FE00E94DB0024
:1008700090E0B0E0A0E07C01DD24CC24FC2A89EDEE
:100880009FE00E94DB00C82F8AED9FE00E94DB0002
:10089000C82ADC2AC092583BD092593BE0925A3B7E
:1008A000F0925B3BCF91FF90EF90DF90CF90089557
:1008B0008091523B882309F48AC08091533B88235E
:1008C00009F485C060915C3B84ED9FE00E94C70005
:1008D0006091180185ED9FE00E94C70060911601AC
:1008E00086ED9FE00E94C7006091583B7091593B94
:1008F00080915A3B90915B3B692F772788279927F6
:1009000087ED9FE00E94C7006091583B7091593B72
:1009100080915A3B90915B3BBC018827992788EDD9
:100920009FE00E94C7006091583B7091593B8091B5
:100930005A3B90915B3B672F782F892F992789ED40
:100940009FE00E94C7006091583B8AED9FE00E94A3
:10095000C7006091543B7091553B8091563B9091FC
:10096000573B692F7727882799278BED9FE00E94B7
:10097000C7006091543B7091553B8091563B9091DC
:10098000573BBC01882799278CED9FE00E94C70048
:100990006091543B7091553B8091563B9091573BF1
:1009A000672F782F892F99278DED9FE00E94C70030
:1009B0006091543B8EED9FE00E94C70063E78FED8E
:1009C0009FE00E94C7008AE090E00C945E018AE0FC
:1009D00090E00C942E0160E08FED9FE00C94C70036
:1009E00082E390E00E94F4000E9461038EE59BE3A5
:1009F0000E9499221092533B08958091543B90910C
:100A0000553BA091563BB091573B892B8A2B8B2BA2
:100A1000E1F08091583B9091593BA0915A3BB091A5
:100A20005B3B892B8A2B8B2B81F080911601909157
:100A300017018F3F910549F080915C3B90915D3BA0
:100A4000892B19F010921501089581E0809315010A
:100A5000089580915101863440F420914F013091E6
:100A6000500181E02E353A4108F080E00895CF939F
:100A70008EE59BE30E94A620C82F0E9478296093F0
:100A80004C3770934D3780934E3790934F37C0FF5C
:100A90002DC081E080935737809356378093553728
:100AA000809150379091513720915737211108C0CC
:100AB00020915637211104C020915537222319F176
:100AC00020910F013091100182179307B0F4019625
:100AD000909351378093503781E0809354378091C1
:100AE00053378823E9F0CF910C94E40010925737E4
:100AF0001092563710925537D3CF81E080935437F8
:100B000080935337ECCF009741F001979093513782
:100B10008093503710925437E2CF10925337FACF68
:100B2000CF910C94E8000F931F930E9478290091B5
:100B30004C3710914D3720914E3730914F37601B15
:100B4000710B820B930B00910B0110910C01209102
:100B50000D0130910E01601771078207930720F095
:100B60001F910F910C9437051F910F9108951092CA
:100B7000900089E18093910088E99CE5909397002B
:100B80008093960080E2809371000895809109011E
:100B9000809347370895803C61F46BED70E080E806
:100BA0009BE30E94DD008CED682F80E89BE30C94B2
:100BB00091268B3DC9F76BED70E080E89BE30E94C6
:100BC000DD008DEDF1CF60EC70E080E89BE30E94EA
:100BD000DD0061E270E080E89BE30E94DD0080912F
:100BE0005F370E94CB0580915E370E94CB058091D4
:100BF0005D370E94CB0580915C370E94CB0560EC8D
:100C000070E080E89BE30C94DD0060EC70E080E82D
:100C10009BE30E94DD0062E270E080E89BE30E94BB
:100C2000DD0080915B370E94CB0580915A370E948E
:100C3000CB05809159370E94CB05809158370E948F
:100C4000CB0560EC70E080E89BE30C94DD00CF9373
:100C5000C0911201C35660EC70E080E89BE30E94F3
:100C6000DD0063E270E080E89BE30E94DD008C2FF2
:100C70000E94CB0560EC70E080E89BE3CF910C9480
:100C8000DD0060EC70E080E89BE30E94DD0064E240
:100C900070E080E89BE30E94DD0080914E3B0E9463
:100CA000CB0560EC70E080E89BE30C94DD0060EC29
:100CB00070E080E89BE30E94DD0062E070E080E885
:100CC0009BE30E94DD0080915B3B0E94CB058091FD
:100CD0005A3B0E94CB058091593B0E94CB058091E5
:100CE000583B0E94CB0560EC70E080E89BE30C94DD
:100CF000DD0060EC70E080E89BE30E94DD0061E0D5
:100D000070E080E89BE30E94DD008091573B0E94E9
:100D1000CB058091563B0E94CB058091553B0E94AC
:100D2000CB058091543B0E94CB0560EC70E080E8DD
:100D30009BE30C94DD00CF93DF93C8E3DFE0CE01AB
:100D40000E94DB000E94CB052196C11580E1D807E7
:100D5000B1F7DF91CF91089560EC70E080E89BE3FC
:100D60000E94DD0061E570E080E89BE30E94DD0009
:100D70000E949B0660EC70E080E89BE30C94DD0031
:100D8000CF93C82F60EC70E080E89BE30E94DD0009
:100D900060E970E080E89BE30E94DD006C2F80E852
:100DA0009BE30E94912660EC70E080E89BE3CF918A
:100DB0000C94DD00CF93DF93C82FD62F0E945703EA
:100DC00081110BC0C83C48F48C2F90E06D2F885CDB
:100DD000904FDF91CF910C94C70083E0DF91CF91CA
:100DE0000C94C0060E94FD048091533B81111DC0EC
:100DF0008091150181113CC08091523B8823C1F143
:100E00004091543B5091553B6091563B7091573BFC
:100E10008EE59BE30E94EC22892B41F481E00E9445
:100E2000C00690E080E00E94F400089581E0809385
:100E3000533B0E94E4020E9416030E94CA020E94D1
:100E4000D7020E9429038EE59BE30E948A2466EE66
:100E50007AE08EE59BE30E942E2270E060E08EE552
:100E60009BE30E94DC2483E090E00E945E01DDCFE2
:100E700083E090E00E942E01D8CF0E945703882380
:100E8000F1F00E9471038823D1F00E947B03882334
:100E9000B1F00E948A03882391F00E94970388236F
:100EA00089F081E08093523B0E94DD03882351F05A
:100EB0000E94E70382E1809314010C94F2061092E1
:100EC000523B08950895CF93DF9380E00E94942BC6
:100ED0000E94E727ACEDBCE1CEE5DAE1FD019E0121
:100EE000119221503040E1F7EAE3F7E3B183A083A8
:100EF000B783A683B583A48389E397E3938382832F
:100F000026E040E052EC61E070E080E89BE30E9464
:100F1000D8260E94B70561E08CE00E94622A61E059
:100F20008DE00E94622AE8E5F9E384EF91E0DF01B9
:100F30009C011D9221503040E1F7E4E5F9E384E0A3
:100F4000DF011D928A95E9F7E2E5F1E0DF019E01FC
:100F50001D9221503040E1F7C6E4DCE188E0DE017B
:100F6000E82F1D92EA95E9F7A0EBBBE1FD01119294
:100F70008A95E9F7E4EDFCE1D183C083D783C6838A
:100F8000D583C48380ED9CE193838283EEE3FCE10F
:100F9000B183A083B783A683B583A4838AE39CE14E
:100FA0009383828322E030E043E050E064E070E02D
:100FB0008EE59BE30E944E20DF91CF910C943D077C
:100FC00060EC70E080E89BE30E94DD0064E070E08C
:100FD00080E89BE30E94DD0060915C3B80E89BE33E
:100FE0000E94912660EC70E080E89BE30C94DD00A9
:100FF00060EC70E080E89BE30E94DD0065E070E05B
:1010000080E89BE30E94DD006091180180E89BE38B
:101010000E94912660EC70E080E89BE30C94DD0078
:1010200060EC70E080E89BE30E94DD0063E070E02C
:1010300080E89BE30E94DD006091160180E89BE35D
:101040000E94912660EC70E080E89BE30C94DD0048
:10105000CF93C82F60EC70E080E89BE30E94DD0036
:1010600060E470E080E89BE30E94DD006C2F80E884
:101070009BE30E94912660EC70E080E89BE3CF91B7
:101080000C94DD00CF93DF9390914937992309F4B5
:1010900041C2803C09F050C080910A0181113CC2DC
:1010A00010924937809151018634A8F580914F0103
:1010B000909150018E359A4170F560914B0170917D
:1010C0004C0180914D0190914E01019710F48DE5F6
:1010D0009AE18617970769F16817790720F5861B4B
:1010E000970BEC0121962097B1F0809151018F5F11
:1010F0008093510184ED9CE10E94AF00BE018EE31C
:101100009CE10E94AF0080914D0190914E0190931F
:101110004C0180934B010E942905811107C2DF9188
:10112000CF910C944602861B970BEC01C15AD54E09
:10113000DACFC1E0D0E0D9CF20914A3730914B3798
:10114000243FF1E03F0708F0F1C190910A01211519
:10115000310529F49E3F19F480930A01E7C19111EA
:1011600046C08B3D21F481E080934837DFC19091E8
:101170004837992349F08C3D21F08D3D19F48BEDD2
:1011800001C080EC1092483790915101963408F0DC
:10119000CDC120914F01309150012E353A4108F0D8
:1011A000C5C120914F01309150012F5F3F4F3093C7
:1011B000500120934F0120914D0130914E01A90122
:1011C0004F5F5F4F50934E0140934D012E5A3E4F5B
:1011D000F901808380914D0190914E018E359A41A5
:1011E00009F0A4C110924E0110924D019FC191309F
:1011F00009F046C08B3DE1F49093483780914A371F
:1012000090914B37049709F091C1609154397091D6
:10121000553980915639909157390E94E22D6115C8
:10122000710581059105E9F4DF91CF910C94790660
:1012300090914837992349F08C3D21F08D3D19F468
:101240008BED01C080EC10924837A9014F5F5F4FD2
:1012500050934B3740934A372C5A364CF9018083D0
:10126000CDCF6093543B7093553B8093563B909306
:10127000573B809114018131B9F60E943A03D4CFD3
:10128000923009F047C08B3DE9F481E08093483704
:1012900080914A3790914B37049709F047C160918C
:1012A00054397091553980915639909157390E942F
:1012B000E22D6115710581059105E9F4DF91CF916A
:1012C0000C94570690914837992349F08C3D21F0B2
:1012D0008D3D19F48BED01C080EC10924837A901C7
:1012E0004F5F5F4F50934B3740934A372C5A364CE1
:1012F000F9018083CDCF6093583B7093593B809325
:101300005A3B90935B3B809114018131B9F60E9466
:101310001603D4CF9330A9F48F3F21F4DF91CF91FE
:101320000C941008823108F081E190E0909317014D
:101330008093160180911401813181F70E94E402AB
:10134000EDCF9430E1F48F3F21F4DF91CF910C94F5
:10135000E007863088F090E08D30910514F08CE045
:1013600090E090935D3B80935C3B809114018131D0
:1013700061F70E94CA02E9CF86E090E0F2CF953093
:10138000E1F48F3F21F4DF91CF910C94F807853081
:1013900088F090E08930910514F088E090E0909317
:1013A00019018093180180911401813161F70E9425
:1013B000D702E9CF85E090E0F2CF963089F48F3FF5
:1013C00021F4DF91CF910C941402811103C00E948B
:1013D000F604F7CF813009F0A9C00E94F206F1CFE0
:1013E000913221F4DF91CF910C94E305923221F4F4
:1013F000DF91CF910C940506933221F4DF91CF91C8
:101400000C942706973031F40E94FD04DF91CF91B0
:101410000C942D02903329F490E0DF91CF910C943D
:101420005E01903431F40E944D03DF91CF910C9412
:101430002808983039F4833709F078C0DF91CF91CC
:101440000C9494029E3069F4813031F48093513BC6
:10145000DF91CF910C9476028111FACF1092513B1B
:10146000F7CF9F3049F40E942905882309F457CE0D
:10147000DF91CF910C945E02993529F4883F09F0F1
:1014800055C00E94F004913521F4DF91CF910C9466
:10149000AC06923569F58B3D91F481E08093483735
:1014A00080914A3790914B37029709F03FC0609185
:1014B000553980915439DF91CF910C94DA0690918F
:1014C0004837992349F08C3D21F08D3D19F48BED7F
:1014D00001C080EC10924837A9014F5F5F4F5093D5
:1014E0004B3740934A372C5A364CF9018083D8CF7A
:1014F000903521F4DF91CF910C94AC02933521F417
:10150000DF91CF910C945804943581F4DF91CF9101
:101510000C94EB04803C51F481E0809349378EEFCA
:1015200080930A0110924B3710924A37DF91CF9186
:1015300008954FB7F89420913E3730913F3780910E
:101540004037909141374FBF2817390711F19FB7A6
:10155000F894E0913E37F0913F3720913C3730913D
:101560003D37E217F30769F420913A3730913B3762
:1015700030933F3720933E3780819FBF0E944208BF
:10158000D8CFE0913E37F0913F379F012F5F3F4F1B
:10159000EFCF0895CF93DF93EC012197A0F08EE574
:1015A0009BE30E94162120914C3B30914D3BA901B9
:1015B0004F5F5F4F50934D3B40934C3B285A364C06
:1015C000F9018083EACFDF91CF9108950F931F93A4
:1015D000CF93DF93EC018091513B8111B5C08EE533
:1015E0009BE30E94162121974091110180FF78C052
:1015F0009C0154E0359527955A95E1F72F703327D4
:101600004F3FD9F410924D3B10924C3B2093110167
:101610008EE59BE30E94BD209093130180931201FD
:101620008EE59BE30E94A92080934E3BCE01DF9183
:10163000CF911F910F910C94CA0A4213E3CF8EE50C
:101640009BE30E94BD202091120130911301820F73
:10165000931F97FD0196959587959093130180931D
:10166000120100914E3B10E08EE59BE30E94A92001
:10167000800F912F911D9595879580934E3BCE01BC
:101680000E94CA0A8FEF809311010E9427060E94D0
:10169000410660EC70E080E89BE30E94DD0070E0B2
:1016A00060E080E89BE30E94DD00C8E5D9E320917B
:1016B0004C3B30914D3BCE0188559943821793079F
:1016C000A0F56991603C39F56BED70E080E89BE333
:1016D0000E94DD006CED80E89BE30E949126E7CF3D
:1016E0004F3F39F010924D3B10924C3B8FEF80935F
:1016F00011018EE59BE30E94BD209093130180931E
:1017000012018EE59BE30E94A92080934E3BCE01FF
:101710000E94CA0ABACF6B3DF1F66BED70E080E82B
:101720009BE30E94DD006DEDD6CF60EC70E080E8B9
:101730009BE30E94DD0010924D3B10924C3BDF91E9
:10174000CF911F910F91089510924D3B10924C3BF9
:101750008EE59BE30E94BD209093130180931201BC
:101760008EE59BE30E94A92080934E3BCE010E9410
:10177000CA0A0E9427060E94410660EC70E080E8D9
:101780009BE30E94DD0070E060E080E89BE30E9444
:10179000DD00C8E5D9E320914C3B30914D3BCE01B3
:1017A000885599438217930708F0BFCF6991603C31
:1017B00061F46BED70E080E89BE30E94DD006CED6E
:1017C00080E89BE30E949126E6CF6B3DC9F76BED65
:1017D00070E080E89BE30E94DD006DEDF1CFCF92D9
:1017E000DF92EF92FF920F931F93CF93DF93EC0161
:1017F0008091533B882309F47AC08091513B811139
:1018000058C00E94EC0060E071E080E090E00E942F
:10181000EF27162F107FCF3FD10508F0116070E041
:1018200060E08EE59BE30E94BB24612F8EE59BE385
:101830000E94082090E6C92E97E3D92EEE24E39467
:10184000F12CC601805697438C179D07F0F4F601E2
:1018500061916F018EE59BE30E940820FFEFEF1A74
:10186000FF0A8FEFE816F10461F78EE59BE30E9413
:10187000B32170E060E08EE59BE30E94BB24612F02
:101880008EE59BE30E940820D9CF8EE59BE30E9462
:10189000B3210E94F00070E060E08EE59BE3DF91F1
:1018A000CF911F910F91FF90EF90DF90CF900C940C
:1018B000DC240E94EC00CF3FD10519F010F0CFEFEF
:1018C000D0E070E060E08EE59BE30E94BB2400E680
:1018D00017E3C801805697438C179D07B0F6F801AF
:1018E00061918F018EE59BE30E940820F2CF82E098
:1018F0000E94C00685E090E0DF91CF911F910F918B
:10190000FF90EF90DF90CF900C94F400EF92FF9255
:101910000F931F93CF93DF9380914A0181116EC083
:1019200081E080934A01D0E0C0E00EE51AE18091A9
:1019300051018C171D0609F008F460C02FB7F89408
:10194000E091D81CF091D91C8091D61C9091D71CA5
:10195000E817F90709F03EC08091D41C9091D51C7E
:101960009093D91C8093D81C808191812FBF4FB751
:10197000F894E091421CF091431C2091401C30915E
:10198000411CE217F30769F520913E1C30913F1C82
:101990003093431C2093421C208131814FBF21157D
:1019A000310551F1E0E6F7E3AC01405657437A01C7
:1019B000CF018056974382179307D8F4C7018E0F43
:1019C0009F1FB8010E94842DDC01AE5ABE4F8C913E
:1019D0008193EECFE091D81CF091D91CCF010296F3
:1019E000BFCFE091421CF091431C9F012E5F3F4FFF
:1019F000CFCFC9010E94EF0B219699CF10925101D0
:101A00001092500110924F0110924A01DF91CF9134
:101A10001F910F91FF90EF900C9446028091533BE1
:101A2000882371F10E94930580915101882311F15F
:101A300080915237811102C00E943705809154373E
:101A400081111AC080915337811116C0809152378D
:101A5000882331F062E370E080E090E00E94A929E1
:101A60000E94370580915437811104C0109252377B
:101A70000E94860C0C94990A81E080935237FACF29
:101A80008091523B882319F00E948A01F3CF0E9473
:101A9000CF010E94F604EECF80E89BE30E94072668
:101AA000892B09F44EC080E89BE30E9421269FB752
:101AB000F89440913E3750913F3720913A3730911A
:101AC0003B374217530769F44091403750914137F3
:101AD00020913C3730913D374217530711F49FBF97
:101AE000DBCF409140375091413720913E373091C4
:101AF0003F37215031094217530789F39FBF2FB752
:101B0000F894E0914037F09141378083409140371D
:101B10005091413780913C3790913D374817590794
:101B200051F480913A3790913B37909341378093AD
:101B300040372FBFD5CF80914037909141370196E4
:101B4000F4CF08951F920F920FB60F9211240BB687
:101B50000F922F933F934F935F936F937F938F9346
:101B60009F93AF93BF93EF93FF930E944C0DFF9110
:101B7000EF91BF91AF919F918F917F916F915F9105
:101B80004F913F912F910F900BBE0F900FBE0F9072
:101B90001F9018952F923F924F925F926F927F9273
:101BA0008F929F92AF92BF92CF92DF92EF92FF926D
:101BB0000F931F93CF93DF93CDB7DEB7C857D109EB
:101BC0000FB6F894DEBF0FBECDBFE9969FAF8EAFC4
:101BD000E9971A01DC0118960D911D912D913C9108
:101BE0001B9761960CAF1DAF2EAF3FAF61971C9650
:101BF0000D911D912D913C911F9709831A832B8381
:101C00003C8350960D911D912D913C9153970D83DE
:101C10001E832F83388754960D911D912D913C91F1
:101C2000579709871A872B873C87E6966FAFE69709
:101C3000E7967FAFE797A85ABF4F6396BFAFAEAFA7
:101C40006397FC01E45AFF4F6596FFAFEEAF6597CF
:101C50008C01005A1F4F67961FAF0EAF67979C010C
:101C60002C593F4F69963FAF2EAF699788599F4FC8
:101C70006B969FAF8EAF6B97E996AEADBFADE99710
:101C8000A459BF4F6D96BFAFAEAF6D97E996EEAD5D
:101C9000FFADE997E059FF4F6F96FFAFEEAF6F973B
:101CA000E9960EAD1FADE9970C581F4FA1961FAFD7
:101CB0000EAFA197E9962EAD3FADE99728583F4F5B
:101CC000A3963FAF2EAFA397E9968EAD9FADE99750
:101CD00084589F4FA5969FAF8EAFA597E996AEAD5E
:101CE000BFADE997A058BF4FA796BFAFAEAFA797BC
:101CF000E996EEADFFADE997EC57FF4FA996FFAF20
:101D0000EEAFA997E9960EAD1FADE99708571F4FA3
:101D1000AB961FAF0EAFAB97E9962EAD3FADE997EF
:101D200024573F4FAD963FAF2EAFAD97E9968EAD9E
:101D30009FADE99780579F4FAF969FAF8EAFAF97FC
:101D4000E996AEADBFADE997AC56BF4FE196BFAFD8
:101D5000AEAFE197E796AEADBFADE7970D911D91A0
:101D60002D913C910D871E872F87388B6396EEADA2
:101D7000FFAD6397008311832283338361968CAD1B
:101D80009DADAEADBFAD619788589B45A549B842A2
:101D9000800F911FA21FB31F4D815E816F817885D7
:101DA00009851A852B853C85402751276227732793
:101DB00009811A812B813C814023512362237323A3
:101DC00009851A852B853C85402751276227732773
:101DD000840F951FA61FB71F8C019D0147E0000FC0
:101DE000111F221F331F4A95D1F7AC01BD01E9E154
:101DF0007695679557954795EA95D1F7402B512BE6
:101E0000622B732B89819A81AB81BC81480F591F4A
:101E10006A1F7B1FE796AEADBFADE79714960D9195
:101E20001D912D913C911797098B1A8B2B8B3C8B15
:101E30006596EEADFFAD65970083118322833383F2
:101E400089859A85AB85BC858A5A9844A843B74151
:101E5000800F911FA21FB31FC980DA80EB80FC8026
:101E60000D811E812F813885C026D126E226F326DA
:101E7000C422D522E622F722C026D126E226F32666
:101E80008C0D9D1DAE1DBF1D8C019D01FCE0000F42
:101E9000111F221F331FFA95D1F76C017D01A4E1B8
:101EA000F694E794D794C794AA95D1F7C02AD12A7B
:101EB000E22AF32AC40ED51EE61EF71EE796AEAD43
:101EC000BFADE79718968D919D910D90BC91A02D77
:101ED0008D8B9E8BAF8BB88F6796EEADFFAD6797FE
:101EE00080839183A283B3838D819E81AF81B885E6
:101EF00085529F48AF4DBB4D0D891E892F89388D66
:101F0000800F911FA21FB31F49805A806B807C8075
:101F100044265526662677264C205D206E207F209D
:101F200009811A812B813C81402651266226732625
:101F3000840D951DA61DB71D8C019D01EFE0369502
:101F4000279517950795EA95D1F72C013D01F1E109
:101F5000440C551C661C771CFA95D1F7402A512A6F
:101F6000622A732A4C0C5D1C6E1C7F1CE796AEAD7A
:101F7000BFADE7971C968D919D910D90BC91A02DC2
:101F8000898F9A8FAB8FBC8F6996EEADFFAD699745
:101F900080839183A283B38389819A81AB81BC8141
:101FA00082519143A244BE43098D1A8D2B8D3C8DE5
:101FB000800F911FA21FB31F8A019B010C251D25B5
:101FC0002E253F25042115212621372104271527F9
:101FD00026273727800F911FA21FB31F4C015D01D9
:101FE0001AE0B694A794979487941A95D1F78C0128
:101FF0009D0186E1000F111F221F331F8A95D1F723
:10200000082919292A293B29040D151D261D371DCC
:10201000E796AEADBFADE79750968D919D910D902F
:10202000BC91A02D8D8F9E8FAF8FB8A36B96EEAD18
:10203000FFAD6B9780839183A283B3838155904FCB
:10204000A348BA40840F951FA61FB71FB701A6016A
:102050004425552566257725402351236223732384
:102060004C255D256E257F25840F951FA61FB71F64
:102070004C015D0147E0880C991CAA1CBB1C4A95C9
:10208000D1F7AC01BD01E9E1769567955795479584
:10209000EA95D1F7482959296A297B29400F511F10
:1020A000621F731FE796AEADBFADE79754968D9153
:1020B0009D910D90BC91A02D89A39AA3ABA3BCA325
:1020C0006D96EEADFFAD6D9780839183A283B38350
:1020D000865D9943A847B84B8C0D9D1DAE1DBF1D55
:1020E00073016201C026D126E226F326C422D5223E
:1020F000E622F722C424D524E624F7248C0D9D1D66
:10210000AE1DBF1D4C015D01FCE0880C991CAA1C92
:10211000BB1CFA95D1F76C017D01A4E1F694E7941C
:10212000D794C794AA95D1F7C828D928EA28FB28BC
:10213000C40ED51EE61EF71EE796AEADBFADE797FF
:1021400058968D919D910D90BC91A02D8DA39EA32D
:10215000AFA3B8A76F96EEADFFAD6F978083918365
:10216000A283B3838D5E994BAF4CB745840D951D0B
:10217000A61DB71D28013901442655266626772657
:102180004C205D206E207F2040265126622673263B
:10219000840D951DA61DB71D4C015D01EFE0B694A1
:1021A000A79497948794EA95D1F72C013D01F1E12A
:1021B000440C551C661C771CFA95D1F74828592801
:1021C0006A287B284C0C5D1C6E1C7F1CE796AEAD0C
:1021D000BFADE7975C968D919D910D90BC91A02D20
:1021E00089A79AA7ABA7BCA7A196EEADFFADA19713
:1021F00080839183A283B3838F5F9A46A94BB240B9
:10220000800F911FA21FB31F8A019B010C251D2562
:102210002E253F25042115212621372104271527A6
:1022200026273727800F911FA21FB31F4C015D0186
:102230001AE0B694A794979487941A95D1F78C01D5
:102240009D0186E1000F111F221F331F8A95D1F7D0
:10225000082919292A293B29040D151D261D371D7A
:10226000E796AEADBFADE79790968D919D910D909D
:10227000BC91A02D8DA79EA7AFA7B8ABA396EEAD3E
:10228000FFADA39780839183A283B383885297463F
:10229000AF47B649840F951FA61FB71FB701A60108
:1022A0004425552566257725402351236223732332
:1022B0004C255D256E257F25840F951FA61FB71F12
:1022C0004C015D0147E0880C991CAA1CBB1C4A9577
:1022D000D1F7AC01BD01E9E1769567955795479532
:1022E000EA95D1F7482959296A297B29400F511FBE
:1022F000621F731FE796AEADBFADE79794968D91C1
:102300009D910D90BC91A02D89AB9AABABABBCABB2
:10231000A596EEADFFADA59780839183A283B3838D
:1023200081559840AB4BB4478C0D9D1DAE1DBF1D14
:1023300073016201C026D126E226F326C422D522EB
:10234000E622F722C424D524E624F7248C0D9D1D13
:10235000AE1DBF1D4C015D01FCE0880C991CAA1C40
:10236000BB1CFA95D1F76C017D01A4E1F694E794CA
:10237000D794C794AA95D1F7C828D928EA28FB286A
:10238000C40ED51EE61EF71EE796AEADBFADE797AD
:1023900098968D919D910D90BC91A02D8DAB9EAB8B
:1023A000AFABB8AFA796EEADFFADA7978083918393
:1023B000A283B3838F54944AA109B109840D951D5A
:1023C000A61DB71D28013901442655266626772605
:1023D0004C205D206E207F204026512662267326E9
:1023E000840D951DA61DB71D4C015D01EFE0B6944F
:1023F000A79497948794EA95D1F72C013D01F1E1D8
:10240000440C551C661C771CFA95D1F748285928AE
:102410006A287B284C0C5D1C6E1C7F1CE796AEADB9
:10242000BFADE7979C968D919D910D90BC91A02D8D
:1024300089AF9AAFABAFBCAFA996EEADFFADA99790
:1024400080839183A283B38382549842A34AB64780
:10245000800F911FA21FB31F8A019B010C251D2510
:102460002E253F2504211521262137210427152754
:1024700026273727800F911FA21FB31F4C015D0134
:102480001AE0B694A794979487941A95D1F78C0183
:102490009D0186E1000F111F221F331F8A95D1F77E
:1024A000082919292A293B29040D151D261D371D28
:1024B000E796AEADBFADE797D0968D919D910D900B
:1024C000BC91A02D21968CAF9DAFAEAFBFAF219731
:1024D000AB96EEADFFADAB9780839183A283B383C0
:1024E0004C015D01FEED8F1AFEEE9F0AFFE6AF0A7A
:1024F000F4E9BF0A840E951EA61EB71EB701A601F9
:1025000044255525662577254023512362237323CF
:102510004C255D256E257F25480D591D6A1D7B1DA7
:102520004A015B0197E0880C991CAA1CBB1C9A9578
:10253000D1F7E9E17695679557954795EA95D1F7F3
:10254000482959296A297B29400F511F621F731F8F
:10255000E796AEADBFADE797D4968D919D910D9066
:10256000BC91A02D25968CAF9DAFAEAFBFAF259788
:10257000AD96EEADFFADAD9780839183A283B3831B
:102580004C015D01FDE68F1AFEE89F0AF7E6AF0AEF
:10259000F2E0BF0A8C0C9D1CAE1CBF1C73016201D3
:1025A000C026D126E226F326C422D522E622F7222F
:1025B000C424D524E624F724C80CD91CEA1CFB1C2F
:1025C00046015701FCE0880C991CAA1CBB1CFA951B
:1025D000D1F7A4E1F694E794D794C794AA95D1F7DC
:1025E000C828D928EA28FB28C40ED51EE61EF71EE7
:1025F000E796AEADBFADE797D8968D919D910D90C2
:10260000BC91A02D29968CAF9DAFAEAFBFAF2997DF
:10261000AF96EEADFFADAF9780839183A283B38376
:102620004C015D01F2E78F1AFCEB9F0AF6E8AF0A56
:10263000F9E5BF0A840C951CA61CB71C28013901BA
:1026400044265526662677264C205D206E207F2066
:102650004026512662267326480C591C6A1C7B1C96
:1026600053014201BFE0B694A79497948794BA951A
:10267000D1F781E1440C551C661C771C8A95D1F773
:10268000482859286A287B284C0C5D1C6E1C7F1C2E
:10269000E796AEADBFADE797DC968D919D910D901D
:1026A000BC91A02D2D968CAF9DAFAEAFBFAF2D9737
:1026B000E196EEADFFADE19780839183A283B38372
:1026C0004C015D01FFED8F1AF7EF9F0AFBE4AF0AA3
:1026D000F6EBBF0A800E911EA21EB31E8A019B015B
:1026E0000C251D252E253F250421152126213721C6
:1026F0000427152726273727080D191D2A1D3B1DDE
:10270000480159019AE0B694A794979487949A95B2
:10271000D1F7E6E1000F111F221F331FEA95D1F711
:10272000082919292A293B29040D151D261D371DA5
:1027300089889A88AB88BC888EE9881A8AED980ABD
:1027400081EEA80A89E0B80A840E951EA61EB71E5F
:10275000B301A20140275127622773274C215D2135
:102760006E217F214425552566257725480D591D65
:102770006A1D7B1D4A015B01F5E0880C991CAA1CAF
:10278000BB1CFA95D1F7ABE17695679557954795C0
:10279000AA95D1F7482959296A297B29400F511F49
:1027A000621F731F8DA09EA0AFA0B8A490EC891AE1
:1027B0009CE4990A9FEBA90A9FE3B90A8C0C9D1C23
:1027C000AE1CBF1C68017901C426D526E626F72673
:1027D000C420D520E620F720C026D126E226F32605
:1027E000C80CD91CEA1CFB1C46015701B9E0880C37
:1027F000991CAA1CBB1CBA95D1F787E1F694E79403
:10280000D794C7948A95D1F7C828D928EA28FB28F5
:10281000C40ED51EE61EF71E89AC9AACABACBCACA0
:10282000AFEA8A1AA5EA9A0AA1EAAA0AA9EDBA0A9F
:10283000840C951CA61CB71C2A013B014C245D246A
:102840006E247F2440225122622273224426552680
:1028500066267726480C591C6A1C7B1C53014201D2
:102860009EE0880C991CAA1CBB1C9A95D1F7E2E14A
:102870007694679457944794EA95D1F74828592855
:102880006A287B284C0C5D1C6E1C7F1C8D849E84EA
:10289000AF84B888B6E58B1AB8E39B0AB9E4AB0AF3
:1028A000B6E1BB0A800E911EA21EB31E97018601DF
:1028B000042515252625372504231523262337230C
:1028C0000C251D252E253F25080D191D2A1D3B1DF4
:1028D00048015901FCE0B694A79497948794FA951F
:1028E000D1F7A4E1000F111F221F331FAA95D1F7C2
:1028F000082919292A293B29040D151D261D371DD4
:1029000089A09AA0ABA0BCA0E3EA8E1AEFEE9E0AC3
:10291000E0EDAE0AE9E2BE0A840E951EA61EB71EC1
:10292000B301A20140275127622773274C215D2163
:102930006E217F214425552566257725480D591D93
:102940006A1D7B1D4A015B01B5E0880C991CAA1C1D
:10295000BB1CBA95D1F78BE176956795579547954E
:102960008A95D1F7482959296A297B29400F511F97
:10297000621F731F8DA89EA8AFA8B8ACFDEA8F1A7E
:10298000FBEE9F0AFBEBAF0AFDEFBF0A8C0C9D1C10
:10299000AE1CBF1C68017901C426D526E626F726A1
:1029A000C420D520E620F720C026D126E226F32633
:1029B000C80CD91CEA1CFB1C4601570199E0880C85
:1029C000991CAA1CBB1C9A95D1F7E7E1F694E794F1
:1029D000D794C794EA95D1F7C828D928EA28FB28C4
:1029E000C40ED51EE61EF71E2D968CAC9DACAEAC6B
:1029F000BFAC2D978FE7881A89E1980A8EE5A80A5F
:102A000087E2B80A840C951CA61CB71C2A013B015E
:102A10004C245D246E247F244022512262227322A2
:102A20004426552666267726480C591C6A1C7B1CB2
:102A300053014201FEE0880C991CAA1CBB1CFA95AC
:102A4000D1F7A2E17694679457944794AA95D1F769
:102A5000482859286A287B284C0C5D1C6E1C7F1C5A
:102A60008D8C9E8CAF8CB8A098E3891A94E0990A5B
:102A70009CE2A90A98E1B90A800E911EA21EB31E1B
:102A800097018601042515252625372504231523BE
:102A9000262337230C251D252E253F25080D191D1E
:102AA0002A1D3B1D48015901BCE0B694A794979498
:102AB0008794BA95D1F784E1000F111F221F331FAD
:102AC0008A95D1F7082919292A293B29040D151DB2
:102AD000261D371D89A89AA8ABA8BCA8AAE18A1A06
:102AE000A2E39A0AAEE1AA0AAEEDBA0A840E951ED6
:102AF000A61EB71EB301A2014027512762277327E4
:102B00004C215D216E217F214425552566257725A1
:102B1000480D591D6A1D7B1D4A015B0195E0880C1B
:102B2000991CAA1CBB1C9A95D1F7EBE17695679589
:102B300057954795EA95D1F7482959296A297B295C
:102B4000400F511F621F731F29968CAC9DACAEAC19
:102B5000BFAC2997BAE28B1AB8EF9B0AB8ECAB0A64
:102B6000BCE3BB0A8C0C9D1CAE1CBF1C6801790128
:102B7000C426D526E626F726C420D520E620F72051
:102B8000C026D126E226F326C80CD91CEA1CFB1C61
:102B900046015701F9E0880C991CAA1CBB1CFA9548
:102BA000D1F7A7E1F694E794D794C794AA95D1F703
:102BB000C828D928EA28FB28C40ED51EE61EF71E11
:102BC000898C9A8CAB8CBC8CE9E78E1AE2EF9E0A5A
:102BD000EAE2AE0AEBE0BE0A840C951CA61CB71C08
:102BE0002A013B014C245D246E247F244022512283
:102BF000622273224426552666267726480C591CE5
:102C00006A1C7B1C53014201BEE0880C991CAA1C63
:102C1000BB1CBA95D1F782E1769467945794479498
:102C20008A95D1F7482859286A287B284C0C5D1CC6
:102C30006E1C7F1C8DA49EA4AFA4B8A8F3E18F1ACC
:102C4000FBEE9F0AF5EAAF0AFAEBBF0A800E911E6F
:102C5000A21EB31E970186010425152526253725BA
:102C600004231523262337230C251D252E253F2538
:102C7000080D191D2A1D3B1D480159019CE0B69401
:102C8000A794979487949A95D1F7E4E1000F111FC8
:102C9000221F331FEA95D1F7082919292A293B2930
:102CA000040D151D261D371D25968CAC9DACAEACB4
:102CB000BFAC25978BEF881A86E1980A8CE1A80AA9
:102CC00086E5B80A840E951EA61EB71EB301A201A2
:102CD00040275127622773274C215D216E217F21D8
:102CE0004425552566257725480D591D6A1D7B1DF0
:102CF0004A015B01F5E0880C991CAA1CBB1CFA95E3
:102D0000D1F7ABE17695679557954795AA95D1F799
:102D1000482959296A297B29400F511F621F731FB7
:102D20008D889E88AF88B88C98E0891A9CE5990AAE
:102D300090E1A90A93E0B90A8C0C9D1CAE1CBF1C43
:102D400068017901C426D526E626F726C420D520B9
:102D5000E620F720C026D126E226F326C80CD91C8F
:102D6000EA1CFB1C46015701B9E0880C991CAA1CFF
:102D7000BB1CBA95D1F787E1F694E794D794C79432
:102D80008A95D1F7C828D928EA28FB28C40ED51E71
:102D9000E61EF71E89A49AA4ABA4BCA4A7E28A1AD3
:102DA000ADEF9A0AA0E9AA0AA8E9BA0A840C951C10
:102DB000A61CB71C2A013B014C245D246E247F24F1
:102DC0004022512262227322442655266626772607
:102DD000480C591C6A1C7B1C530142019EE0880C64
:102DE000991CAA1CBB1C9A95D1F7E2E176946794D2
:102DF00057944794EA95D1F7482859286A287B28A0
:102E00004C0C5D1C6E1C7F1C4601570184249524CC
:102E1000A624B72421968CAD9DADAEADBFAD219754
:102E20008657934BA54DB247800F911FA21FB31F2A
:102E30009501840104231523262337230C251D2502
:102E40002E253F25800F911FA21FB31F8C019D01CE
:102E5000FCE03695279517950795FA95D1F7E596F5
:102E60000CAF1DAF2EAF3FAFE5978C019D01A4E1E4
:102E7000000F111F221F331FAA95D1F7E5968CADC5
:102E80009DADAEADBFADE597082B192B2A2B3B2B83
:102E9000040D151D261D371D89A19AA1ABA1BCA14A
:102EA0008E5B964CA540B109840F951FA61FB71FD6
:102EB00080269126A226B326880E991EAA1EBB1E26
:102EC000D501C40144E0880F991FAA1FBB1F4A9572
:102ED000D1F75CE1B694A794979487945A95D1F76B
:102EE000882A992AAA2ABB2A800E911EA21EB31EE6
:102EF0004DA55EA56FA578A94F5759406E487847F4
:102F00004C0D5D1D6E1D7F1D73016201C026D12613
:102F1000E226F326C824D924EA24FB24C40ED51EB5
:102F2000E61EF71EB701A601EBE0440F551F661F12
:102F3000771FEA95D1F7F5E1F694E794D794C79413
:102F4000FA95D1F7C42AD52AE62AF72AC80CD91C43
:102F5000EA1CFB1C49AD5AAD6BAD7CAD4E5D5E49C4
:102F600062467249440E551E661E771EB901A801BD
:102F7000482559256A257B254C255D256E257F250D
:102F8000440E551E661E771ED20123013D014C0CD6
:102F90005D1C6E1C7F1C29964CAD5DAD6EAD7FAD8A
:102FA0002997445F574C6A417240400F511F621F7E
:102FB000731F950184010C251D252E253F25042511
:102FC000152526253725040F151F261F371FB90184
:102FD000A801A9E07695679557954795AA95D1F7E9
:102FE000B7E1000F111F221F331FBA95D1F7042B31
:102FF000152B262B372B040D151D261D371D498932
:103000005A896B897C894C5B554161447B45480DED
:10301000591D6A1D7B1D4601570184249524A62451
:10302000B72480269126A226B326840E951EA61EBE
:10303000B71EB501A40184E0440F551F661F771F1A
:103040008A95D1F79CE1B694A794979487949A9522
:10305000D1F7842A952AA62AB72A800E911EA21E8D
:10306000B31E4D8D5E8D6F8D78A1475550436142E3
:10307000744BC40ED51EE61EF71EB301A2014027F5
:10308000512762277327482559256A257B254C0D32
:103090005D1D6E1D7F1DDB01CA01EBE0880F991FCE
:1030A000AA1FBB1FEA95D1F7F5E17695679557956D
:1030B0004795FA95D1F7482B592B6A2B7B2B480D56
:1030C000591D6A1D7B1DC9A4DAA4EBA4FCA4B0EAB7
:1030D000CB1AB4EBDB0AB4E4EB0AB9E0FB0A4C0C04
:1030E0005D1C6E1C7F1C68017901C824D924EA2468
:1030F000FB24C426D526E626F7264C0C5D1C6E1C48
:103100007F1CF20123013F01440E551E661E771EEF
:10311000CDA8DEA8EFA8F8ACF0E9CF1AF3E4DF0AF7
:10312000F0E4EF0AF1E4FF0AC00ED11EE21EF31E26
:1031300095018401042715272627372704251525FF
:10314000262537250C0D1D1D2E1D3F1D68017901FB
:10315000A9E0F694E794D794C794AA95D1F7B7E17C
:10316000000F111F221F331FBA95D1F70C291D29FB
:103170002E293F29040D151D261D371D2596CCAC83
:10318000DDACEEACFFAC25978AE3C81A81E8D80A1B
:1031900084E6E80A87EDF80AC80CD91CEA1CFB1C77
:1031A0004A015B0184249524A624B7248026912615
:1031B000A226B3268C0C9D1CAE1CBF1C750164019D
:1031C00084E0CC0CDD1CEE1CFF1C8A95D1F79CE141
:1031D000B694A794979487949A95D1F78C289D28B4
:1031E000AE28BF28800E911EA21EB31ECD84DE84A1
:1031F000EF84F88896E0C91A98EDD90A9EE5E90AA5
:1032000095E1F90AC40ED51EE61EF71EB301A20110
:103210004027512762277327482559256A257B2592
:103220004C0D5D1D6E1D7F1D6A017B01EBE0CC0C1A
:10323000DD1CEE1CFF1CEA95D1F7F5E1769567954C
:1032400057954795FA95D1F74C295D296E297F2925
:10325000480D591D6A1D7B1DC98CDA8CEB8CFC8CCA
:10326000ABE7CA1AAFECDA0AA0E1EA0AABE2FA0A63
:103270004C0C5D1C6E1C7F1C68017901C824D9248C
:10328000EA24FB24C426D526E626F7264C0C5D1C32
:103290006E1C7F1CF20123013F01440E551E661E69
:1032A000771ECDA0DEA0EFA0F8A4FBEFCF1AF2EEC0
:1032B000DF0AF7E7EF0AFBEFFF0AC00ED11EE21E9E
:1032C000F31E950184010427152726273727042597
:1032D0001525262537250C0D1D1D2E1D3F1D6801AA
:1032E0007901A9E0F694E794D794C794AA95D1F709
:1032F000B7E1000F111F221F331FBA95D1F70C2918
:103300001D292E293F29040D151D261D371DC9A86D
:10331000DAA8EBA8FCA887ECC81A8FE2D80A8BE2DF
:10332000E80A86E2F80AC80CD91CEA1CFB1C4A0110
:103330005B0184249524A624B72480269126A22606
:10334000B3268C0C9D1CAE1CBF1C7501640184E06F
:10335000CC0CDD1CEE1CFF1C8A95D1F79CE1B694C9
:10336000A794979487949A95D1F78C289D28AE2896
:10337000BF28800E911EA21EB31E2196CCACDDACE0
:10338000EEACFFAC21979BE1C91A96E6D90A94E20C
:10339000E90A99E1F90AC40ED51EE61EF71EB3012B
:1033A000A2014027512762277327482559256A25FE
:1033B0007B254C0D5D1D6E1D7F1D6A017B01EBE0C1
:1033C000CC0CDD1CEE1CFF1CEA95D1F7F5E17695DF
:1033D000679557954795FA95D1F74C295D296E2940
:1033E0007F29480D591D6A1D7B1D2D96CCACDDAC87
:1033F000EEACFFAC2D97A8E0CA1AA3E8DA0AADE557
:10340000EA0AA0EEFA0A4C0C5D1C6E1C7F1C6801D7
:103410007901C824D924EA24FB24C426D526E6262B
:10342000F7264C0C5D1C6E1C7F1CF20123013F0132
:10343000440E551E661E771ECD88DE88EF88F88CF8
:10344000FBE9CF1AF9EADF0AF3E5EF0AFBE3FF0A2B
:10345000C00ED11EE21EF31E95018401042715271C
:103460002627372704251525262537250C0D1D1D54
:103470002E1D3F1D68017901A9E0F694E794D794C9
:10348000C794AA95D1F7B7E1000F111F221F331F70
:10349000BA95D1F70C291D292E293F29040D151D98
:1034A000261D371DCD84DE84EF84F8888CEBC81A86
:1034B0008DEDD80A86EDE80A8BE0F80AC80CD91C15
:1034C000EA1CFB1C4A015B0180949094A094B09488
:1034D000802A912AA22AB32A84249524A624B724D8
:1034E0008C0C9D1CAE1CBF1C7501640186E0CC0CCD
:1034F000DD1CEE1CFF1C8A95D1F79AE1B694A794C7
:10350000979487949A95D1F78C289D28AE28BF2848
:10351000800E911EA21EB31EC9A4DAA4EBA4FCA4C3
:1035200099E6C91AD10895EDE90A9CEBF90AC40E8F
:10353000D51EE61EF71EB301A20140955095609579
:103540007095482959296A297B29402751276227E4
:1035500073274C0D5D1D6E1D7F1D6A017B01EAE026
:10356000CC0CDD1CEE1CFF1CEA95D1F7F6E176953C
:10357000679557954795FA95D1F74C295D296E299E
:103580007F29480D591D6A1D7B1D2996CCACDDACE9
:10359000EEACFFAC2997A9E5CA1AACEDDA0AABE6A6
:1035A000EA0AA4E5FA0AC40CD51CE61CF71C28019B
:1035B00039014094509460947094442A552A662AA4
:1035C000772A482459246A247B244C0C5D1C6E1CE9
:1035D0007F1C73016201AFE0CC0CDD1CEE1CFF1CF4
:1035E000AA95D1F7B1E17694679457944794BA9528
:1035F000D1F74C285D286E287F28440E551E661E84
:10360000771EC9A0DAA0EBA0FCA0B7ECCB1ABFE5EF
:10361000DB0ABCE6EB0AB3E0FB0AC00ED11EE21ED9
:10362000F31E95018401009510952095309504298D
:1036300015292629372904271527262737270C0D72
:103640001D1D2E1D3F1D680179018BE0F694E79446
:10365000D794C7948A95D1F795E1000F111F221FC7
:10366000331F9A95D1F70C291D292E293F29040DC6
:10367000151D261D371D2196CCACDDACEEACFFAC84
:103680002197EDE3CE1AE6EADE0AE4EAEE0AEAE979
:10369000FE0AC80CD91CEA1CFB1C4A015B01809481
:1036A0009094A094B094802A912AA22AB32A8424C8
:1036B0009524A624B7248C0C9D1CAE1CBF1C750140
:1036C0006401E6E0CC0CDD1CEE1CFF1CEA95D1F792
:1036D000FAE1B694A79497948794FA95D1F78C2839
:1036E0009D28AE28BF28800E911EA21EB31EC98C35
:1036F000DA8CEB8CFC8CFEE6CF1AF3E3DF0AF3EFF7
:10370000EF0AF0E7FF0AC40ED51EE61EF71EB3014E
:10371000A2014095509560957095482959296A29CC
:103720007B2940275127622773274C0D5D1D6E1D95
:103730007F1D6A017B01AAE0CC0CDD1CEE1CFF1C86
:10374000AA95D1F7B6E17695679557954795BA95BD
:10375000D1F74C295D296E297F29480D591D6A1D15
:103760007B1DCDA8DEA8EFA8F8AC83E8C81A8BE0D3
:10377000D80A80E1E80AF108C40CD51CE61CF71C45
:10378000280139014094509460947094442A552A39
:10379000662A772A482459246A247B244C0C5D1C11
:1037A0006E1C7F1C730162018FE0CC0CDD1CEE1CD3
:1037B000FF1C8A95D1F791E17694679457944794CA
:1037C0009A95D1F74C285D286E287F28440E551E07
:1037D000661E771EC988DA88EB88FC889FE2C91AC2
:1037E00092EAD90A9BE7E90A9AE7F90AC00ED11EC4
:1037F000E21EF31E950184010095109520953095E9
:10380000042915292629372904271527262737278C
:103810000C0D1D1D2E1D3F1D68017901EBE0F69476
:10382000E794D794C794EA95D1F7F5E1000F111FFB
:10383000221F331FFA95D1F70C291D292E293F2964
:10384000040D151D261D371DCDA4DEA4EFA4F8A878
:10385000A1EBCA1AA1E8DA0AA7E5EA0AA0E9FA0A7E
:10386000C80CD91CEA1CFB1C4A015B018094909493
:10387000A094B094802A912AA22AB32A8424952461
:10388000A624B7248C0C9D1CAE1CBF1C75016401C2
:10389000A6E0CC0CDD1CEE1CFF1CAA95D1F7BAE10A
:1038A000B694A79497948794BA95D1F78C289D28BD
:1038B000AE28BF28800E911EA21EB31E2D968CAD81
:1038C0009DADAEADBFAD2D9780529941A34DB14096
:1038D000840F951FA61FB71FB301A20140955095F5
:1038E00060957095482959296A297B2940275127D5
:1038F00062277327840F951FA61FB71F6C017D01D8
:103900004AE0CC0CDD1CEE1CFF1C4A95D1F7AC0143
:10391000BD01E6E17695679557954795EA95D1F70C
:103920004C295D296E297F29480D591D6A1D7B1D73
:103930008DA19EA1AFA1B8A58C5E9C4BAE4FBC459E
:10394000840D951DA61DB71D280139014094509482
:1039500060947094442A552A662A772A4824592468
:103960006A247B24840D951DA61DB71D6C017D0165
:10397000FFE0CC0CDD1CEE1CFF1CFA95D1F72C01EE
:103980003D01A1E17694679457944794AA95D1F7A5
:103990004C285D286E287F28440E551E661E771E13
:1039A00025968CAD9DADAEADBFAD25978F559E4E86
:1039B000A74FB14B800F911FA21FB31F9501840128
:1039C0000095109520953095042915292629372929
:1039D0000427152726273727800F911FA21FB31F03
:1039E0006C017D011BE0F694E794D794C7941A9577
:1039F000D1F78C019D0185E1000F111F221F331F9C
:103A00008A95D1F70C291D292E293F29040D151D52
:103A1000261D371D8D8D9E8DAF8DB8A18E57914877
:103A2000AC4AB840880D991DAA1DBB1D4A015B0117
:103A300080949094A094B094802A912AA22AB32AC8
:103A400084249524A624B724880D991DAA1DBB1D86
:103A50006C017D01E6E0CC0CDD1CEE1CFF1CEA9540
:103A6000D1F74C015D01FAE1B694A794979487943D
:103A7000FA95D1F78C289D28AE28BF28800E911E7C
:103A8000A21EB31E89AD9AADABADBCAD8B5C9D40A3
:103A9000A54CB244840F951FA61FB71FB301A20106
:103AA0004095509560957095482959296A297B2938
:103AB0004027512762277327840F951FA61FB71F22
:103AC0006C017D014AE0CC0CDD1CEE1CFF1C4A950C
:103AD000D1F7AC01BD01E6E176956795579547951D
:103AE000EA95D1F74C295D296E297F29480D591D8A
:103AF0006A1D7B1D8D899E89AF89B88D85549D4235
:103B0000A842B54D840D951DA61DB71D280139018C
:103B10004094509460947094442A552A662A772AD7
:103B2000482459246A247B24840D951DA61DB71DA5
:103B30006C017D01FFE0CC0CDD1CEE1CFF1CFA9536
:103B4000D1F72C013D01A1E17694679457944794F5
:103B5000AA95D1F74C285D286E287F28440E551E63
:103B6000661E771E89A99AA9ABA9BCA98F569C424B
:103B7000A947B441800F911FA21FB31F9501840173
:103B80000095109520953095042915292629372967
:103B90000427152726273727800F911FA21FB31F41
:103BA0006C017D011BE0F694E794D794C7941A95B5
:103BB000D1F78C019D0185E1000F111F221F331FDA
:103BC0008A95D1F70C291D292E293F29040D151D91
:103BD000261D371D61968CAD9DADAEADBFAD619715
:103BE000880D991DAA1DBB1D61968CAF9DAFAEAF10
:103BF000BFAF619789819A81AB81BC81800F911F92
:103C0000A21FB31F89839A83AB83BC830D811E815E
:103C10002F813885040D151D261D371D0D831E832C
:103C20002F83388789859A85AB85BC85840F951F3E
:103C3000A61FB71F89879A87AB87BC87E796AEAD6B
:103C4000BFADE797A05CBF4FE796BFAFAEAFE797BA
:103C5000B0E42B1A310811F00C94AA0E61960CAD49
:103C60001DAD2EAD3FAD6197E996AEADBFADE99705
:103C700018960D931D932D933C931B9709811A81E0
:103C80002B813C811C960D931D932D933C931F9784
:103C90000D811E812F81388550960D931D932D9394
:103CA0003C93539709851A852B853C8554960D9333
:103CB0001D932D933C935797E7968EAD9FADE79755
:103CC000C858DF4F0FB6F894DEBF0FBECDBFDF91EF
:103CD000CF911F910F91FF90EF90DF90CF90BF9009
:103CE000AF909F908F907F906F905F904F903F909C
:103CF0002F900895CF93DF93FC0181E093E2A5E438
:103D0000B7E680879187A287B38789E89BEAADEC05
:103D1000BFEE84879587A687B7878EEF9CEDAAEBC9
:103D2000B8E9808B918BA28BB38B86E794E5A2E3F5
:103D3000B0E1848B958BA68BB78B10821182128297
:103D400013821482158216821782DF01A85ABF4F90
:103D500080E4ED01982F19929A95E9F77896DF01A2
:103D60001D928A95E9F7DF91CF9108958F929F92E6
:103D7000AF92BF92EF92FF920F931F93CF93DF9377
:103D8000EC017B018A0188819981AA81BB8170E065
:103D900060E04A015B01880E991EAA1EBB1E2FE13E
:103DA000B22288829982AA82BB8288169906AA06C4
:103DB000BB0668F48C809D80AE80BF802FEF821A96
:103DC000920AA20AB20A8C829D82AE82BF828F734F
:103DD0009927AA27BB270097A105B10579F120E40F
:103DE000822E912CA12CB12C881A990AAA0ABB0AFE
:103DF00048968C0F9D1F481559056A057B0570F480
:103E0000A801B701DF91CF911F910F91FF90EF9023
:103E1000BF90AF909F908F900C94702FA401B7012A
:103E20000E94702FE80CF91C0819190940E450E0B1
:103E3000BE01685E7F4FCE010E94CA0D003411059D
:103E400048F0A801407CB701CE010E94CA0D7C0158
:103E50000F731127A801B701CE014896D3CFEF9277
:103E6000FF920F931F93CF93DF938C01EB01488157
:103E700059816A817B814F73552766277727DB013C
:103E8000CA010196A11DB11D4C0F5D1F20E8FA016A
:103E9000208F40E450E060E070E0481B590B6A0B53
:103EA0007B0B7E01F8E1EF0EF11C483051056105F6
:103EB0007105A0F4489670E060E08C0F9D1F0E9491
:103EC000792F40E450E0B701CE010E94CA0D40E4D2
:103ED00050E060E070E080E090E0DC014850510983
:103EE000489670E060E08C0F9D1F0E94792F8881BA
:103EF0009981AA81BB8123E0880F991FAA1FBB1F4C
:103F00002A95D1F788839983AA83BB83FE01E05B5E
:103F1000FF4F8083319690833196A0833196B08392
:103F20003C812D819E818F81319630833196208313
:103F3000319690833196808340E450E0B701CE0102
:103F40000E94CA0D8885F8018083898581838A85CE
:103F500082838B8583838C8584838D8585838E8501
:103F600086838F85878388898087898981878A89E5
:103F700082878B8983878C8984878D8985878E89C1
:103F800086878F89878788E9FE0111928A95E9F7EC
:103F9000DF91CF911F910F91FF90EF900895CF92F5
:103FA000DF92EF92FF920F931F93CF93DF93CDB7E2
:103FB000DEB7C859D1090FB6F894DEBF0FBECDBF2A
:103FC0007C016B0180E190E00E9409288C01CE0108
:103FD00001960E947A1EA601B701CE0101960E94A9
:103FE000B61EBE016F5F7F4FC8010E942F1FC80120
:103FF000C856DF4F0FB6F894DEBF0FBECDBFDF91BE
:10400000CF911F910F91FF90EF90DF90CF90089587
:10401000CF93DF931F92CDB7DEB76983DC01ED91BB
:10402000FC910280F381E02D41E050E0BE016F5F22
:104030007F4F09950F90DF91CF9108950895FC016E
:104040001382128288EE93E0A0E0B0E0848395832F
:10405000A683B7838BE291E09183808380E5848798
:1040600081E085878AE090E09787868789E090E005
:10407000918B808B82E090E0938B828B148A158ADF
:10408000168A178A118E108E138E128E158E148E2C
:1040900040E050E0BA01CF010C943A27FC01778749
:1040A0006687518B408B338B228B08950F931F9320
:1040B000CF93DF93EC01062F142F60E08E850E94D2
:1040C0009E2A3C852D8580917E3B882381F09FB779
:1040D000F89480917E3B813081F58DB380937C3B59
:1040E0004DB380917D3B809584238DBB9FBF3CBDAC
:1040F0002DBD0EBD00000DB407FEFDCF8EB51EBD5B
:1041000000000DB407FEFDCF1EB580917E3B8823D5
:1041100051F09FB7F89420917E3B80917C3B2130F9
:1041200079F48DBB9FBF61E08E850E949E2A812F0E
:10413000DF91CF911F910F91089590937C3BD7CF42
:104140008FBFF1CF6F7740E00C94562068E10C945C
:10415000A22069E10C94A22069E10E94A220682FAC
:10416000880F770B880B990B0E94672C20E030E0BA
:1041700040E85EE30E94172D08958F929F92AF92C0
:10418000BF92EF92FF920F931F93CF93DF938C0117
:104190006AE10E94A220C82FD0E0C8010E94AC2092
:1041A0000E942F2C4B017B01F80164897589868957
:1041B00097890E94672C24ED30E843E45EE40E9476
:1041C0002A2CBE0187FD12C06D597109F7FE11C07E
:1041D000680D791DCB01DF91CF911F910F91FF9059
:1041E000EF90BF90AF909F908F900895645A71099F
:1041F000EDCF072E000C880B990B0E94672C20EB4B
:1042000032E748E85FE30E94172D0E942F2CE2CF8F
:10421000CF93DF93EC0163E10E94A22090E0288D10
:10422000398D821B930BDF91CF910895CF93DF934C
:10423000EC01E881F9810480F581E02D0995892B55
:1042400069F0888D998D0196998F888F60E0CE01F5
:104250000E94A22090E0DF91CF9108958FEF9FEF11
:10426000FACF0F931F93CF93DF938C0166E00E94E8
:10427000A220D82F67E0C8010E94A220C82F68E0C2
:10428000C8010E94A2204C2F50E070E060E0762F21
:10429000652F542F44276D2B8A019B01082BC901E0
:1042A000B80120E038E448EE51E00E94F42D03E12B
:1042B0000E94992EB901CA01DF91CF911F910F91F0
:1042C00008956DE10E94A220E82FF0E084E0F595CA
:1042D000E7958A95E1F7EA30F10508F036C0ED5828
:1042E000FE4D0C94D92DA6217D21AB218221872161
:1042F0008C21912196219B21A02160EA78E280E027
:1043000090E0089560E471E580E090E0089562E156
:104310007AE780E090E0089564EE72EA80E090E051
:10432000089564E274EF80E090E0089568E478EE28
:1043300081E090E0089560E970ED83E090E00895F9
:1043400060E271EA87E090E00895089568E77EE111
:1043500080E090E0089560EF7CE380E090E00895D5
:104360006CE20C94A220CF93DF93EC0143E861E868
:104370000E94562062E1CE010E94A22083FD03C06C
:104380000E94CC2AF7CF48E062E9CE010E94562075
:1043900081E090E0DF91CF910895AF92BF92CF92EC
:1043A000DF92FF920F931F93CF93DF936C015B011A
:1043B000EA0162E20E94A220F82E90E09C012C0FFC
:1043C0003D1F2F3F310529F020F0CFEFD0E0C81B73
:1043D000D90B8501AC0EBD1E0A151B0541F0F80175
:1043E00041918F0160E8C6010E945620F5CF4C2F05
:1043F0004F0D62EAC6010E945620CE01DF91CF9197
:104400001F910F91FF90DF90CF90BF90AF900895D4
:104410000F931F93CF93DF93EC01E881F981048020
:10442000F581E02D0995892BB1F06DE0CE010E9458
:10443000A220082F60E0CE010E94A220182F402F5A
:104440006DE8CE010E945620812F90E0DF91CF9140
:104450001F910F9108958FEF9FEFF8CFCF93DF93C8
:10446000EC017D8F6C8F8A899B89672BA1F160E0BD
:104470000E94622A40E060ECCE010E9456208A89A8
:104480009B8982309105D9F08A309105D1F00B9744
:10449000D1F481E00E94A0258A899B898230910510
:1044A000A1F08A30910599F00B9799F481E043E0EF
:1044B00050E062E375E2DF91CF910C94CE2A82E066
:1044C000E9CF80E0E7CF8FEFE5CF82E0F0CF80E06B
:1044D000EECF8FEFECCF82309105B9F08A309105A5
:1044E000B1F00B97B1F481E00E94FD2A8A899B8983
:1044F0008230910581F08A30910579F00B9779F43B
:1045000081E0DF91CF910C94BF2582E0EDCF80E078
:10451000EBCF8FEFE9CF82E0F4CF80E0F2CF8FEFE7
:10452000F0CF41E861E80C94562040E861E80C9433
:1045300056200E9495220C948C25AF92BF92CF9268
:10454000DF92EF92FF920F931F93CF93DF93EC01D3
:10455000DB01CA018C8B9D8BAE8BBF8B6A017B010B
:10456000FF0CCC08DC2C76019A01AB016C2D7C2D64
:104570008C2D9C2D03E10E947E2EA12CE8E4BE2E02
:10458000F8EECF2EDD24D394E12CF12C00E010E0E6
:104590000E94212E122FC22ED32E7A01A701662748
:1045A000772766E8CE010E94562077276F2D5E2D73
:1045B0004D2D67E8CE010E945620412F68E8CE01BC
:1045C000DF91CF911F910F91FF90EF90DF90CF90EF
:1045D000BF90AF900C945620CF92DF92EF92FF9253
:1045E000CF93DF93EC016A017B0161E08E850E942D
:1045F000622A61E08E850E949E2A888999898F3F70
:104600009807B9F061E00E94622A60E088890E9400
:104610009E2A6AE070E080E090E00E94A92961E0B3
:1046200088890E949E2A6AE070E080E090E00E9403
:10463000A9290E94562562E4CE010E94A22082315F
:1046400091F5CE010E949522B701A601CE010E94EC
:104650009D2240E06EE8CE010E94562040E06FE8C7
:10466000CE010E9456206CE0CE010E94A220482F6D
:1046700043606CE8CE010E94562044E066EACE0119
:104680000E94562040E869E8CE010E945620CE01E3
:104690000E94912281E090E0DF91CF91FF90EF9016
:1046A000DF90CF90089590E080E0F6CFCF92DF9238
:1046B000EF92FF92CF93DF93EC016EE10E94A22074
:1046C000F82ECE010E946121F2942FE0F222CC2438
:1046D000C394D12C02C0CC0CDD1CFA94E2F70D2C53
:1046E000000CEE08FF0828EE33E040E050E00E94A6
:1046F000BA2DC701B6010E94BA2D213131054105FD
:1047000051055CF04CE066EACE01DF91CF91FF905D
:10471000EF90DF90CF900C94562044E0F4CF0F93AD
:104720001F93CF93DF938C01EB016630710534F05A
:104730006D30710534F56630710529F545EC61EB96
:10474000C8010E9456204CE067EBC8010E94562029
:10475000C6E0D0E06EE1C8010E94A2208F7094E014
:10476000CC0FDD1F9A95E1F74C2F482B6EE9C8015D
:104770000E945620C801DF91CF911F910F910C9498
:104780005623CCE0D0E043EC61EBC8010E945620F8
:104790004AE067EBC8010E945620DCCFCF92DF923F
:1047A000EF92FF920F931F93CF93DF938C01CB0176
:1047B000BA010E94672C6B017C0120E030EC43EFD2
:1047C00055E40E942A2CD0E0C0E018160CF065C019
:1047D00020E030E842E256E4C701B6010E942A2CEC
:1047E000C1E0D0E018160CF058C020E030EC43E7F0
:1047F00056E4C701B6010E942A2CC2E0D0E0181688
:104800000CF04BC020E030E842EA56E4C701B601A4
:104810000E942A2CC3E0D0E018160CF03EC020E025
:1048200034E244EF56E4C701B6010E942A2CC4E0EA
:10483000D0E0181694F520E034EE42E257E4C701C8
:10484000B6010E942A2CC5E0D0E0181634F520E00D
:1048500034E244E757E4C701B6010E942A2CC6E0BF
:10486000D0E01816D4F420E034E244EF57E4C70156
:10487000B6010E942A2CC7E0D0E0181674F420E09C
:1048800034E244E758E4C701B6010E942A2CC9E08B
:10489000D0E0181614F0C8E0D0E06DE1C8010E9425
:1048A000A2208F7094E0CC0FDD1F9A95E1F74C2F7A
:1048B000482B6DE9C8010E945620C801DF91CF91B5
:1048C0001F910F91FF90EF90DF90CF900C945623A3
:1048D0000F931F93CF93DF938C01EB016930710528
:1048E00014F0C8E0D0E06DE1C8010E94A220C530FC
:1048F000D10514F4C5E0D0E02497CC0FDD1F482F7C
:10490000417F4C2B6DE9C801DF91CF911F910F9131
:104910000C945620CF93DF93EC016EE10E94A2200D
:10492000482F44606EE9CE01DF91CF910C94562060
:10493000CF93DF93EC011B8E1A8E6DE10E94A220B3
:10494000482F4E7F6DE9CE01DF91CF910C94562018
:10495000CF93DF93EC0181E090E09B8F8A8F6DE134
:10496000CE010E94A220482F41606DE9CE01DF9167
:10497000CF910C9456200F931F93CF93DF93EC01AC
:104980008B010E949122CE01012B99F00E94A82454
:1049900040E06DE8CE010E94562040E062EACE0180
:1049A0000E94562081E090E0DF91CF911F910F91FE
:1049B00008950E949824ECCF0F931F93CF93DF9319
:1049C000EC018B011616170684F40E94A824402FD0
:1049D00062EACE010E94562045E861E8CE01DF91EF
:1049E000CF911F910F910C9456200E949824F4CFE0
:1049F0000F931F93CF93DF93EC0162E10E94A220FB
:104A0000182F482F62E9CE010E94562015FD25C0BF
:104A1000198E188E8A8D9B8D62E2892B09F463E1D1
:104A2000CE010E94A220082F10E060E1CE010E947A
:104A3000A220482F6DE8CE010E945620EC8DFD8DFE
:104A4000309711F0C801099540E06DE8CE01DF9183
:104A5000CF911F910F910C945620DF91CF911F9110
:104A60000F9108958EE59BE30C94F824452B61F497
:104A7000AB016F30710514F04EE050E057FD40E09F
:104A8000406769E80C945620AB016231710514F05F
:104A900041E150E04230510514F442E050E0425010
:104AA0004068EFCF8EE59BE30C941F20CF93CFB7E8
:104AB000F89480917F3B811127C0E0EDF0E0849174
:104AC000E0EBF0E09491E82FF0E0EE0FFF1FEA50EA
:104AD000FF4FA591B491EC91E92321F461E084E0CA
:104AE0000E949E2A61E084E00E94622A8CB5806167
:104AF0008CBD8CB580648CBD61E087E00E94622A29
:104B000061E085E00E94622A80917F3B8F5F809305
:104B10007F3BCFBFCF9108959FB7F89480917F3BA3
:104B2000882319F0815080937F3B80917F3B8111D6
:104B300005C08CB58F7B8CBD10927E3B9FBF0895C6
:104B40002FB7F894813041F0C0F08230A1F082E0BC
:104B500080937E3B80E001C082E090917D3B892B79
:104B600080937D3B80917E3B811103C081E08093E7
:104B70007E3B2FBF089584E0F0CF81E0EECF90918F
:104B80007E3B9230A1F09FB7F894833088F4E82FF1
:104B9000F0E0E95CFE4F8081809520917D3B82238F
:104BA00080937D3B811102C010927E3B9FBF089590
:104BB00080E0F2CFAF92BF92CF92DF92EF92FF925E
:104BC0000F931F93CF93DF936C017B018B01040F35
:104BD000151FEB015E01AE18BF08C017D10759F0D1
:104BE0006991D601ED91FC910190F081E02DC60113
:104BF0000995892B79F7C501DF91CF911F910F910D
:104C0000FF90EF90DF90CF90BF90AF900895FC01A0
:104C1000918D228D892F90E0805C9F4F821B91099E
:104C20008F7399270895FC01918D828D981731F02B
:104C3000828DE80FF11D858D90E008958FEF9FEF35
:104C40000895FC01918D828D981761F0A28DAE0FB1
:104C5000BF2FB11D5D968C91928D9F5F9F73928F38
:104C600090E008958FEF9FEF089580EA97E2892BF7
:104C700049F080E090E0892B29F00E94A027811163
:104C80000E94000080E090E0892B49F080E090E0F5
:104C9000892B29F00E94000081110C9400000895D6
:104CA000FC01A48DA80FB92FB11DA35ABF4F2C91A1
:104CB000848D90E001968F739927848FA689B78998
:104CC0002C93A089B1898C9180648C93938D848D71
:104CD000981306C00288F389E02D80818F7D808340
:104CE0000895CF93DF93EC01888D8823B9F0AA89CA
:104CF000BB89E889F9898C9185FD03C0808186FD97
:104D00000DC00FB607FCF7CF8C9185FFF2CF8081E5
:104D100085FFEDCFCE010E945026E9CFDF91CF91E4
:104D20000895EF92FF920F931F93CF93DF93EC01BF
:104D300081E0888F9B8D8C8D981316C0E889F98946
:104D4000808185FF11C0EE89FF896083E889F98938
:104D500080818064808381E090E0DF91CF911F911A
:104D60000F91FF90EF900895F62E0B8D10E00F5FDE
:104D70001F4F0F731127E02E8C8D8E110CC00FB6B4
:104D800007FCFACFE889F989808185FFF5CFCE014C
:104D90000E945026F1CFEB8DEC0FFD2FF11DE35A51
:104DA000FF4FF0820B8FEA89FB8980818062D2CF2E
:104DB000CF92DF92EF92FF921F93CF93DF93EC019C
:104DC0006A017B01122FE889F98982E08083C1148E
:104DD00081EED806E104F104A1F060E079E08DE312
:104DE00090E0A70196010E94982D215031094109B8
:104DF00051095695479537952795211580E1380734
:104E000098F0E889F989108260E874E88EE190E012
:104E1000A70196010E94982D21503109410951099D
:104E20005695479537952795EC85FD853083EE851A
:104E3000FF852083188EEC89FD891083EA89FB8920
:104E4000808180618083EA89FB898081886080839A
:104E5000EA89FB89808180688083EA89FB89808177
:104E60008F7D8083DF91CF911F91FF90EF90DF9036
:104E7000CF900895FC01448355836683778308951A
:104E80001F920F920FB60F9211240BB60F922F9311
:104E90008F939F93EF93FF93E091903BF091913B21
:104EA0008081E091963BF091973B82FD1DC09081FF
:104EB0008091993B8F5F8F7320919A3B821741F0CD
:104EC000E091993BF0E0E058F44C958F8093993B4A
:104ED000FF91EF919F918F912F910F900BBE0F90AB
:104EE0000FBE0F901F9018958081F2CF1F920F92E6
:104EF0000FB60F9211240BB60F922F933F934F933F
:104F00005F936F937F938F939F93AF93BF93EF9331
:104F1000FF9380E89BE30E945026FF91EF91BF91A1
:104F2000AF919F918F917F916F915F914F913F9141
:104F30002F910F900BBE0F900FBE0F901F901895E2
:104F400080E89BE30E94072621E0892B09F420E0FA
:104F5000822F0895E0E8FBE31382128288EE93E04B
:104F6000A0E0B0E084839583A683B7838EE391E0CD
:104F70009183808385EC90E09587848784EC90E032
:104F80009787868780EC90E0918B808B81EC90E016
:104F9000938B828B82EC90E0958B848B86EC90E0F7
:104FA000978B868B118E128E138E148E0895089512
:104FB0000E94E2290E94D7270E946307C5E3D6E238
:104FC0000E940E0D2097E1F30E943526F9CF00973D
:104FD00029F0BC0190E080E00C94672F0895CF92F7
:104FE000DF92EF92FF926B017C01C114D104E104C6
:104FF000F10441F00E94182FA70196010E94BA2DDA
:105000006B017C01C701B601FF90EF90DF90CF905C
:1050100008950F931F93CF93DF938230910510F47F
:1050200082E090E0E091283CF091293C30E020E0E3
:10503000B0E0A0E0309799F42115310509F44AC099
:10504000281B390B24303105D8F58A819B816115E5
:10505000710589F1FB0193838283FE0111C04081B8
:1050600051810281138148175907E0F04817590709
:1050700099F4109761F012960C93129713961C9363
:105080003296CF01DF91CF911F910F910895009338
:10509000283C1093293CF4CF2115310551F04217DB
:1050A000530738F0A901DB019A01BD01DF01F801C6
:1050B000C1CFEF01F9CF9093293C8093283CCDCF0D
:1050C000FE01E20FF31F819391932250310939833E
:1050D0002883D7CF2091263C3091273C232B41F4C5
:1050E00020911C0130911D013093273C2093263CD8
:1050F00020911A0130911B012115310541F42DB782
:105100003EB740911E0150911F01241B350BE091C9
:10511000263CF091273CE217F307A0F42E1B3F0B2F
:105120002817390778F0AC014E5F5F4F2417350719
:1051300048F04E0F5F1F5093273C4093263C8193CD
:1051400091939FCFF0E0E0E09CCFCF93DF93009767
:10515000E9F0FC01329713821282A091283CB091B1
:10516000293CED0130E020E01097A1F4208131814D
:10517000820F931F2091263C3091273C2817390736
:1051800009F061C0F093273CE093263CDF91CF917A
:105190000895EA01CE17DF07E8F54A815B819E0199
:1051A00041155105B1F7E901FB83EA834991599112
:1051B000C40FD51FEC17FD0761F480819181029621
:1051C000840F951FE90199838883828193819B8352
:1051D0008A83F0E0E0E012968D919C9113970097FE
:1051E000B9F52D913C911197CD010296820F931F35
:1051F0002091263C3091273C2817390739F6309703
:1052000051F51092293C1092283CB093273CA09372
:10521000263CBCCFD383C28340815181840F951F2C
:10522000C817D90761F44E5F5F4F88819981480F95
:10523000591F518340838A819B81938382832115E7
:10524000310509F0B0CFF093293CE093283C9ECF84
:10525000FD01DC01C0CF13821282D7CF1F920F92C3
:105260000FB60F9211242F933F938F939F93AF9379
:10527000BF9380911E3C90911F3CA091203CB09127
:10528000213C30911D3C23E0230F2D3758F501962A
:10529000A11DB11D20931D3C80931E3C90931F3C8B
:1052A000A093203CB093213C8091223C9091233CE0
:1052B000A091243CB091253C0196A11DB11D809385
:1052C000223C9093233CA093243CB093253CBF9177
:1052D000AF919F918F913F912F910F900FBE0F90A3
:1052E0001F90189526E8230F0296A11DB11DD2CF5D
:1052F0002FB7F89460911E3C70911F3C8091203C28
:105300009091213C2FBF08953FB7F8948091223CA3
:105310009091233CA091243CB091253C26B5A89BBC
:1053200005C02F3F19F00196A11DB11D3FBFBA2F37
:10533000A92F982F8827BC01CD01620F711D811DF7
:10534000911D42E0660F771F881F991F4A95D1F77C
:1053500008958F929F92AF92BF92CF92DF92EF9279
:10536000FF926B017C010E9484294B015C01C114F6
:10537000D104E104F104E9F00E94CC2A0E948429BE
:10538000681979098A099B09683E7340810591056E
:1053900070F321E0C21AD108E108F10888EE880E06
:1053A00083E0981EA11CB11CC114D104E104F104D6
:1053B00029F7FF90EF90DF90CF90BF90AF909F9034
:1053C0008F900895789484B5826084BD84B581609F
:1053D00084BD85B5826085BD85B5816085BDEEE6FD
:1053E000F0E0808181608083E1E8F0E010828081DC
:1053F00082608083808181608083E0E8F0E080814A
:1054000081608083E1EBF0E0808184608083E0EB69
:10541000F0E0808181608083E1E9F0E0808182605A
:105420008083808181608083E0E9F0E08081816019
:105430008083EAE7F0E080818460808380818260FD
:1054400080838081816080838081806880831092E6
:10545000C100089581508A3080F5E82FF0E0ED5CBE
:10546000F54D0C94D92D472A4B2A3D2A432A5D2A13
:105470005D2A4E2A542A582A5E2A809180008F770E
:10548000809380000895809180008F7DF9CF84B54E
:105490008F7784BD089584B58F7DFBCF8091B00058
:1054A0008F778093B00008958091B0008F7DF9CF01
:1054B000809190008F778093900008958091900064
:1054C0008F7DF9CFCF93DF9390E0FC01E455FF4F40
:1054D000249184539F4FFC0184918823C9F090E06C
:1054E000880F991FFC01EA50FF4FA591B491FC0170
:1054F000E451FF4FC591D49161110DC09FB7F8944D
:105500008C91209582238C938881282328839FBFA8
:10551000DF91CF910895623051F49FB7F8943C9198
:10552000822F809583238C93E8812E2BEFCF8FB72A
:10553000F894EC912E2B2C938FBFEACF1F93CF932F
:10554000DF93282F30E0F901E457FF4F8491F901F0
:10555000E455FF4FD491F901E453FF4FC491CC239C
:10556000A9F0162F81110E942A2AEC2FF0E0EE0FED
:10557000FF1FE451FF4FA591B4918FB7F894EC91C0
:10558000111108C0D095DE23DC938FBFDF91CF913E
:105590001F910895DE2BF8CF08950895833060F5AC
:1055A000E82FF0E0EE0FFF1FE05EFE4F7183608397
:1055B000813051F08230A1F0809169008C7F482BBE
:1055C00040936900E89A089580916900837F440FB1
:1055D000551F440F551F482B40936900E99A0895C1
:1055E000809169008F7C94E0440F551F9A95E1F7F4
:1055F000482B40936900EA9A0895833078F4E82FA5
:10560000F0E0813061F0823061F0E898EE0FFF1F2A
:10561000E05EFE4F8DEC9AE2918380830895E998D5
:10562000F5CFEA98F3CF1F920F920FB60F92112485
:105630000BB60F922F933F934F935F936F937F938C
:105640008F939F93AF93BF93EF93FF93E0912001CC
:10565000F09121010995FF91EF91BF91AF919F9139
:105660008F917F916F915F914F913F912F910F900B
:105670000BBE0F900FBE0F901F9018951F920F92A8
:105680000FB60F9211240BB60F922F933F934F93A7
:105690005F936F937F938F939F93AF93BF93EF939A
:1056A000FF93E0912201F09123010995FF91EF9181
:1056B000BF91AF919F918F917F916F915F914F912A
:1056C0003F912F910F900BBE0F900FBE0F901F9028
:1056D00018951F920F920FB60F9211240BB60F92CE
:1056E0002F933F934F935F936F937F938F939F93EA
:1056F000AF93BF93EF93FF93E0912401F0912501C5
:105700000995FF91EF91BF91AF919F918F917F91FB
:105710006F915F914F913F912F910F900BBE0F9022
:105720000FBE0F901F901895883020F0873108F435
:1057300087E188512091260190E4299F900111244E
:105740008770822B80937C0080917A0080648093A4
:105750007A0080917A0086FDFCCF8091780090914C
:10576000790008951F93CF93DF93182FEB0161E029
:105770000E94622A209739F460E0812FDF91CF9157
:105780001F910C949E2ACF3FD10511F461E0F5CF13
:10579000E12FF0E0E457FF4FE491E150EA3008F0E8
:1057A00054C0F0E0EA52F44D0C94D92DE02BE82BD4
:1057B000ED2BF72B252C252C012C092C112C1B2C27
:1057C00084B5806884BDC7BDDF91CF911F910895D6
:1057D00084B5806284BDC8BDF7CF809180008068A9
:1057E00080938000D0938900C0938800EDCF809192
:1057F0008000806280938000D0938B00C0938A00E9
:10580000E3CF8091B00080688093B000C093B30074
:10581000DBCF8091B00080628093B000C093B40071
:10582000D3CF80919000806880939000D0939900AE
:10583000C0939800C9CF80919000806280939000BF
:10584000D0939B00C0939A00BFCFC038D1050CF015
:105850009DCF92CF0E94A22C08F481E008950E946F
:10586000362C6894B1110C94112D08950E94F62CD9
:1058700088F09F5798F0B92F9927B751B0F0E1F011
:10588000660F771F881F991F1AF0BA95C9F714C0C1
:10589000B13091F00E94102DB1E008950C94102DBC
:1058A000672F782F8827B85F39F0B93FCCF38695FA
:1058B00077956795B395D9F73EF490958095709557
:1058C00061957F4F8F4F9F4F0895E89409C097FBD4
:1058D0003EF490958095709561957F4F8F4F9F4FC7
:1058E0009923A9F0F92F96E9BB279395F69587950B
:1058F00077956795B795F111F8CFFAF4BB0F11F4CE
:1059000060FF1BC06F5F7F4F8F4F9F4F16C0882374
:1059100011F096E911C0772321F09EE8872F762FAA
:1059200005C0662371F096E8862F70E060E02AF0EB
:105930009A95660F771F881FDAF7880F96958795D7
:1059400097F90895990F0008550FAA0BE0E8FEEFAC
:1059500016161706E807F907C0F012161306E40733
:10596000F50798F0621B730B840B950B39F40A262C
:1059700061F0232B242B252B21F408950A2609F40A
:10598000A140A6958FEF811D811D089597F99F670E
:1059900080E870E060E008959FEF80EC08950024B7
:1059A0000A941616170618060906089500240A9484
:1059B00012161306140605060895092E0394000C0A
:1059C00011F4882352F0BB0F40F4BF2B11F460FF99
:1059D00004C06F5F7F4F8F4F9F4F089557FD9058C2
:1059E000440F551F59F05F3F71F04795880F97FBA3
:1059F000991F61F09F3F79F087950895121613065D
:105A00001406551FF2CF4695F1DF08C0161617068B
:105A10001806991FF1CF86957105610508940895C0
:105A2000E894BB2766277727CB0197F908950E9452
:105A30002A2D0C94DD2C0E94CF2C38F00E94D62CFD
:105A400020F0952311F00C94C62C0C94CC2C11242E
:105A50000C94112D0E94EE2C70F3959FC1F3950FBD
:105A600050E0551F629FF001729FBB27F00DB11DE2
:105A7000639FAA27F00DB11DAA1F649F6627B00D72
:105A8000A11D661F829F2227B00DA11D621F739F5B
:105A9000B00DA11D621F839FA00D611D221F749F69
:105AA0003327A00D611D231F849F600D211D822FB0
:105AB000762F6A2F11249F5750409AF0F1F08823D7
:105AC0004AF0EE0FFF1FBB1F661F771F881F915004
:105AD0005040A9F79E3F510580F00C94C62C0C94C1
:105AE000112D5F3FE4F3983ED4F386957795679543
:105AF000B795F795E7959F5FC1F7FE2B880F911D2E
:105B00009695879597F90895AA1BBB1B51E107C08D
:105B1000AA1FBB1FA617B70710F0A61BB70B881F3D
:105B2000991F5A95A9F780959095BC01CD010895CC
:105B3000A1E21A2EAA1BBB1BFD010DC0AA1FBB1F91
:105B4000EE1FFF1FA217B307E407F50720F0A21B03
:105B5000B30BE40BF50B661F771F881F991F1A9470
:105B600069F760957095809590959B01AC01BD019A
:105B7000CF010895052E97FB1EF400940E94D12DAD
:105B800057FD07D00E94982D07FC03D04EF40C94CB
:105B9000D12D50954095309521953F4F4F4F5F4FF8
:105BA000089590958095709561957F4F8F4F9F4F89
:105BB0000895EE0FFF1F0024001C0BBE0790F69106
:105BC000E02D099469279627692778278727782762
:105BD00008950E94B42EA59F900DB49F900DA49F90
:105BE000800D911D11240895E894DF93CF93FC015B
:105BF000DB010E94B42E7F936F93E9019A01AC01FF
:105C0000BF93AF933F932F93DF010E94B42E26F4EE
:105C10006C1B7D0B820B930B9E01EB01FC010E9420
:105C2000C32EAF91BF912F913F910E94C32EBE0111
:105C3000CF01F9012F913F91CF91DF9108956894A1
:105C400001C0E8948F929F92CF93DF930E942D2EF4
:105C5000DF91CF919F908F90089588249924F4012B
:105C6000E401B0E49F93AA279A158B049C04ED05E8
:105C7000FE05CF05D007A10798F4AD2FDC2FCF2F5D
:105C8000FE2FE92D982C892E982F872F762F652FA0
:105C9000542F432F322F2227B85031F7BF9127C0FE
:105CA0001B2EBF91BB27220F331F441F551F661F9A
:105CB000771F881F991F881C991CEE1FFF1FCC1F80
:105CC000DD1FAA1FBB1F8A149B04EC05FD05CE0532
:105CD000DF05A007B10748F08A189B08EC09FD0909
:105CE000CE09DF09A00BB10B21601A94E1F62EF466
:105CF0009401AF01BE01CD01000C0895002E0830C3
:105D000090F0982F872F762F652F542F432F322F07
:105D100022270850F4CF220F331F441F551F661F40
:105D2000771F881F991F0A95B2F7002D089597FDD8
:105D30001094002E083098F00850232F342F452F50
:105D4000562F672F782F892F912DF4CF1594979583
:105D500087957795679557954795379527950A9530
:105D6000AAF71124002D0895A29FB001B39FC0018E
:105D7000A39F700D811D1124911DB29F700D811D77
:105D80001124911D08950E94B42E460F571FC81F5D
:105D9000D91F08F4319608958F929F92AF92BF92C7
:105DA000CF92DF92EF92FF92CF93DF93EC01688165
:105DB00079818A819B81611571058105910521F4A5
:105DC00064E279ED8BE597E02DE133EF41E050E0BF
:105DD0000E94BA2D49015A019B01AC01A7EAB1E426
:105DE0000E94E92D6B017C01ACEEB4EFA50194019A
:105DF0000E94992FC60ED71EE81EF91EF7FE06C098
:105E000081E0C81AD108E10880E8F80AC882D9827E
:105E1000EA82FB82C701B6019F77DF91CF91FF90A5
:105E2000EF90DF90CF90BF90AF909F908F900895AC
:105E30008F929F92AF92BF92CF92DF92EF92FF929A
:105E40006091000170910101809102019091030124
:105E5000611571058105910521F464E279ED8BE509
:105E600097E02DE133EF41E050E00E94BA2D490167
:105E70005A019B01AC01A7EAB1E40E94E92D6B0134
:105E80007C01ACEEB4EFA50194010E94992FC60EDF
:105E9000D71EE81EF91EF7FE06C081E0C81AD10819
:105EA000E10880E8F80AC0920001D0920101E09276
:105EB0000201F0920301C701B6019F77FF90EF90B6
:105EC000DF90CF90BF90AF909F908F900895609398
:105ED00000017093010180930201909303010895E2
:105EE000FB01DC0102C001900D9241505040D8F7F7
:105EF0000895DC0101C06D9341505040E0F70895D2
:105F0000F999FECF92BD81BDF89A992780B5089581
:105F1000262FF999FECF1FBA92BD81BD20BD0FB6C5
:105F2000F894FA9AF99A0FBE01960895B7FF0C9467
:105F3000E92D0E94E92D821B930B0895F894FFCF61
:105F400001000000F82A00002801FE030000000FF5
:105F500000FFDCFE1101FF00050000002A3C80006C
:105F6000CD2ACD2ACD2A01000000000820CD21082D
:105F700021162108221E20010204000000009126A3
:0A5F8000DA250726212613267126D4
:00000001FF
